:020000009D2839
:08000800002882073334333471
:100010003234203406340C34013402342008820790
:100020000034013402340334043405340634073414
:10003000083409340A340B340C340D340E340F34C4
:100040008207522BF32BE82C572C7C2B112C1B2DC9
:10005000842CA32B292C382DA82CCA2B402C532DB3
:10006000C82C8207DF2A142B442A382B82075334EA
:100070007434613474346E34233431342034233492
:1000800032342034233433342034233434340034B1
:100090008207533465347234763420344D346F34EF
:1000A0006434653420345034613467342F3452342E
:1000B000673400348207203445346D34653472343B
:1000C000673465346E346334793420345334743493
:1000D0006F3470342134003482074D3469346E3407
:1000E00069344434433443342034533474346134F5
:1000F000743469346F346E342034003482075634DB
:1001000065347234733469346F346E34203435346A
:100110002E34343400348207543472346E346F34E5
:100120007534743420344334743472346C34203471
:100130004D346F34643465340034BF208E2533274A
:10014000D408031DB2284327A626A926AC26AF262D
:100150004327DC26E026E426E826641847225618C2
:100160004722A02833274327BB20D4080319A328FC
:10017000D6184722B3284626C1193C260800073066
:100180009F0083162C308500860183128601213062
:1001900084006030A0008001840AA00BCB28463088
:1001A0008400B701370887258000840AB70A063023
:1001B0003706031DD228B2229030CC00CD00CE00ED
:1001C000CF008030D700D900F830D800DA00DD0A3F
:1001D0004130E1000800C1180800D408031D0800E0
:1001E000C1140430AE0056180800D40AC0303026BE
:1001F000B70137085A20B70A003E0319012918260B
:10020000F9284A08A800CA01C3224208EA004308A4
:10021000EB004408EC004508ED004130C200C3008B
:10022000C400C5006E1CC216EE1CC3166E1DC4169B
:10023000EE1DC5160A30A5001930B700B927851D77
:100240003B294327A626A926AC26AF264327A50B84
:100250001C292808CA0056106A08C2006B08C3008F
:100260006C08C4006D08C500C322B225F625D40170
:10027000C0304B23F62DC0304B23C110D4012808C9
:10028000CA004229C1180800C1140430AE00B222CD
:100290005408D40A3128D6196A293522D615D4250E
:1002A000C03030264C3084000430BA002D300018A5
:1002B0002A3018262D3080182A3018262D300019A3
:1002C0002A3018262D3080192A301826840ABA0BB5
:1002D00056290800D601D401B225F62DDF0ADF0A1F
:1002E000DF0ADF0ADF0ADF0ADF0ADF0ADF0A600847
:1002F000DB00DC00DB0DDB0DDB0D5C0D5B075F075E
:10030000CB0058105A105F08E000DF010800803071
:1003100030265230182665301826633018269C295E
:10032000561C0800D6190800803030265030182698
:100330006C30182679301826312752301826743040
:1003400018266530182631276108182631275D08E0
:10035000262631274B087F3926267C30CB1B2F30B1
:100360001826E62956190800DD0A04305D076707DC
:100370008725A90803195615CB0008005611DD0B77
:10038000B529DD0A080061085A3A03190800E10A94
:10039000CF296108413A03190800E103CF2956111A
:1003A000E701413061020319DF29E80005306707E2
:1003B0008725E70AA908031DD629E80BD6290130AD
:1003C000DD00053067078725CB0008007B30E9009A
:1003D000B4000530B20032088725A908031DE903DF
:1003E000B20AB40BEB29C03030265B3018266908FE
:1003F0002A265D30182ECB0803190E2A5818CB1761
:1004000004305D076707EA008725A908031917224A
:100410004B08A2006A086E255611B22904305D0708
:100420006707EA008725A908031D262208006A0835
:10043000803CEB008030E5006508E5036508872512
:10044000A200650A6E25EB0B1D2A08006A08803C95
:10045000EB006A08E5006508E50A65088725A20043
:1004600065036E25EB0B2C2AB529B5010130182642
:10047000342EC1180800C1140430AE00561C412AA5
:100480004B293522561490293522D6148729641811
:10049000652A59085702031D502A5A085802031D9D
:1004A0005422D61C902987295708D9005808DA0009
:1004B00055275708BD00B900622789275808BE0094
:1004C000B9006227BF01C0016F2FE608031D6C2A27
:1004D00005306707E500DD01E60A6608323A031DCC
:1004E0000800E601E60A65088725E50AA908031958
:1004F000832ADD0A7B2ACB00A91F812AAF2243274A
:10050000502A89227F2A6410E601DD080319DD0ADA
:1005100008005810CB134B08033EDB00D701D71758
:10052000D81058110310DB0C0318D8140310DB0C7F
:10053000031858150310DB0C031857140310DB0CB9
:100540000318D7140310DB0C031857150310DB0C2A
:100550000318D7150310DB0C03185716080058149E
:10056000CB178B2A60304A1A8030C2006030CA1A1A
:100570008030C30060304A1B8030C4006030CA1B2A
:100580008030C500EE01E030C205C305C405C505D5
:100590004A1C4216CA1C43164A1D4416CA1D45165B
:1005A00080304A1AC205CA1AC3054A1BC405CA1BB1
:1005B000C505D001D101D201D301AD0108008030C1
:1005C0003026B70137083620B70A003E0319EA2A59
:1005D0001826E22AC030302641301826643018260A
:1005E000643018267230182620304A1C3C304A1AD3
:1005F0003E301826460826262030CA1C3C30CA1A2F
:100600003E3018264708262620304A1D3C304A1B1B
:100610003E301826480826262030CA1D3C30CA1B0A
:100620003E3018264908262E80303026B70137087C
:100630004820B70A003E03191F2B1826172BD20A91
:10064000C030302643301826563018263A30182647
:100650002D08AC005008013E2A262D3018265108DE
:100660002A263127520826262D3018265308262EF2
:10067000B222D401B701D601463084000008A2009E
:1006800037086E25840AB70A05303706031D3E2B4E
:100690003522B225F62D30261030D5003127D50B66
:1006A0004E2B0800D619792B5618752BD618782B97
:1006B000D408031D622B10304A1A602B4A1CC20654
:1006C000CC060800D4180800541C08004C164A1820
:1006D0006D2B4A1A6F2B4A16EA2A4A10712B4A12BE
:1006E0004A1442124A1C4216EA2A6414E60108001F
:1006F000FB290830CC065029D619A02B56189F2B61
:10070000D6189F2BD408031D8C2B1030CA1A8A2BA5
:10071000CA1CC306CD060800D4180800541C0800E3
:100720004D16CA18972BCA1A992BCA16EA2ACA104C
:100730009B2BCA12CA144312CA1C4316EA2AC9299F
:100740000830CD065029D619C72B5618C62BD618F7
:10075000C62BD408031DB32B10304A1BB12B4A1DE6
:10076000C406CE060800D4180800541C08004E1613
:100770004A19BE2B4A1BC02B4A17EA2A4A11C22B20
:100780004A134A1544124A1D4416EA2AC32908305E
:10079000CE065029D619F02B5618ED2BD618ED2B76
:1007A000D408031DDA2B1030CA1BD82BCA1DC5066E
:1007B000CF060800D4180800541C08004F16CA19A8
:1007C000E52BCA1BE72BCA17EA2ACA11E92BCA1361
:1007D000CA154512CA1D4516EA2A5818892AAF2A91
:1007E0000830CF065029D6190E2C56180D2CD618C5
:1007F0000D2CD418022C20304A1A8030C206013049
:10080000EE06080033275208B100EC263327FE26F7
:1008100033270130B100EC26332FBE290430CC063B
:100820005029D619262C5618252CD618252CD41824
:10083000202C2030CA1A8030C3060230EE06080091
:1008400033275008D300FE26332F6E290430CD06FF
:100850005029D6193D2C56183C2CD6183C2CD418AF
:10086000382C20304A1B8030C4060430EE060800C5
:10087000332728272827332F71290430CE06502903
:10088000D619542C5618532CD618532CD4184F2C38
:100890002030CA1B8030C5060830EE06080033271A
:1008A00010271027332F74290430CF065029D6196A
:1008B000812C5618802CD618802C5418712CD418E2
:1008C000742C1F304A1C0F304A1A7F30500603190F
:1008D0000800D00A4A1C6F2C1030C206421EC20A01
:1008E0000800C60AEA220800D00AFF3050060319A1
:1008F000AD0AD30A53197D2C202BD301D20A202B09
:10090000B2290130CC065029D619A52C5618A42C92
:10091000D618A42C54189E2CD418A12C1F30CA1CF5
:100920000F30CA1A7F30510603190800D10ACA1CB9
:100930009C2C1030C306431EC30A0800C70AEA22D3
:100940000800D10A202B080070290130CD0650295B
:10095000D619C52C5618C42CD618C42C5418C22C21
:10096000D41808001F304A1D0F304A1B7F30520632
:1009700003190800D20A4A1DC02C1030C406441EB8
:10098000C40A0800C80AEA2A73290130CE06502991
:10099000D619E52C5618E42CD618E42C5418E22C61
:1009A000D41808001F30CA1D0F30CA1B7F305306F1
:1009B00003190800D30ACA1DE02C1030C506451ED5
:1009C000C50A0800C90AEA2A76290130CF0650294B
:1009D000D619182D5618172DD618172D5418FD2C6A
:1009E000D418002D500803190800D0034A1CFB2C12
:1009F0001030C206421AC2030800C603EA220800E9
:100A0000D30353190D25D003FE3050060319AD034F
:100A1000FF302D0603191125202B0330D300D203FC
:100A200008000230AD07D3008030D20008007729DB
:100A30000230CC065029D619352D5618342DD6182B
:100A4000342D5418302DD418322D510803190800B4
:100A5000D103CA1C2E2D1030C306431AC30308004D
:100A6000C703EA2AD103202B6F290230CD06502973
:100A7000D619502D56184F2DD6184F2D54184D2DD0
:100A8000D4180800520803190800D2034A1D4B2D40
:100A90001030C406441AC4030800C803EA2A7229A5
:100AA0000230CE065029D6196B2D56186A2DD6184D
:100AB0006A2D5418682DD41808005308031908002B
:100AC000D3031030CA1D662DC506451AC50308009C
:100AD000C903EA2A75290230CF065029A6008725C6
:100AE000220603190800260883169B001C158B1389
:100AF0008312220883169A0055309D00AA309D006B
:100B00009C149C18812D1C118B17831208008316CE
:100B10009B001C141A088312A90008003426B70190
:100B2000B501370805201826B70AB71D912D3426C0
:100B30009C25CD27B225F62D80303026B701370809
:100B40006C20B70A003E0319A72D18269F2DC03030
:100B50003026B70137087E20B70A003E0319080087
:100B60001826AA2D803030264C3018266F301826D3
:100B7000633018263A301826460826262D304C1A9F
:100B80002A301826470826262D304D1A2A301826D6
:100B9000480826262D304E1A2A30182649082626BF
:100BA0002D304F1A2A30182E803030264C3018261F
:100BB000460826262D304C1A2A3018264C30182686
:100BC000470826262D304D1A2A3018264C30182674
:100BD000480826262D304E1A2A3018264C30182662
:100BE000490826262D304F1A2A30182EC0303026BC
:100BF0007E306E187F30182650082A267E30EE1878
:100C00007F30182651082A267E306E197F3018262C
:100C100052082A267E30EE197F30182653082A2ED5
:100C2000B400340E0F393038182634080F393038F4
:100C3000B2001430A300A30B1B2E1E26B20E3208E6
:100C40000F3935048600851485100800BC009827EC
:100C50002A08102EBC009827280816262A08102ECD
:100C600035121826351608001430A3009630B70048
:100C7000C127A30B362E08002F082020C111D4084D
:100C8000031D080056180800B225F62D051D4E2E2E
:100C90008519522ED408031D4229392AD408031D70
:100CA0004229EB28C11C5C2EAE0B0800C11032306B
:100CB000AE000C30E20008009526EF30A4000608D4
:100CC0000B10A40C031C7E2E2408860000000B1CB5
:100CD0005F2E4118752E4114060EA7008026AF0026
:100CE000C1140430AE00C1159F2EAE0B9F2E0C30E8
:100CF0006202031DE2036208AE00732E4110742EDF
:100D0000A001A41D8A2EA00A241D8A2EA00AA41CBC
:100D10008A2EA00A271C0E28A71C932E271D912E71
:100D20002015A0150E2820150E280608B600FF3045
:100D3000860083168113F03086008312080036087F
:100D40008600831681178601831208005527B22674
:100D5000BD2E5527B426C12E5527B626C52E55279C
:100D6000B826C92E4608B92E4708B92E4808B92E0C
:100D70004908BD00B9006227892F42084A1AD22EBD
:100D8000CC2E4308CA1AD22ECC2E44084A1BD22E8F
:100D9000CC2E4508CA1BD22EBE00B9006227BF0167
:100DA000C0016F2FBF003F30BE00B9006227892706
:100DB0003F08B9006227D02E5527B2264C08CC2E0A
:100DC0005527B4264D08CC2E5527B6264E08CC2ED6
:100DD0005527B8264F08CC2E0630B30053277D3058
:100DE000B900BD00622789273108BE00B90062271B
:100DF000BF01C0016F27B30BEE2E08000630B30011
:100E0000532753087F397838B900BD0062278927F6
:100E10005108BE00B90062276F27B30B002F0800EE
:100E20005527B901BD0162278927EC30BE002D1876
:100E30003E14AD18BE14B900622789275008BF00C0
:100E4000B900622789275108C000B90062276F2FB7
:100E50005327BE017C30BD002D183D14AD18BD14C4
:100E60001B2F2030182E1430B2005527B901BD01B8
:100E7000BE0162278927B9016227BF01C0016F2720
:100E8000B20B352F08005527FF30B900BD0062278F
:100E9000492F4A2F4B2F00008927B901BE01622735
:100EA000BF01C0016F2F1930562F0F30A300582FEC
:100EB000592F00007E27A30B572F5E2F5F2F602F27
:100EC0000000892F0830BB000310B91F6D2F7E274B
:100ED000692FB90DBB0B652F08008927692F89275A
:100EE0003D083E063F064006B90062277E27BF0147
:100EF000C001D4080319BB20892F08007F2F0330BD
:100F0000B700C1279527842F00000430B700C12700
:100F1000952F8A2F00000730B700C127952708308A
:100F2000912F922FB700C127952F01308506080019
:100F300003101030BA00A501A801AA01BC0DAC0D28
:100F4000AA0DA80DA50DBA0BA62F00342A30AD2787
:100F50002830AD272530AD279E2F840003300007B1
:100F6000A100A119800030300007A100A11B800062
:100F700000343708D500C8303708C127D50BBB2F40
:100F800000340000C32FC42F0130B8000000C82F68
:100F9000B80BC62FB70BC42F00340A30A50032306F
:0A0FA000B700B927A50BCF2F0800FA
:02400E00303F41
:1042000003000400050006000F000000000000008D
:10421000000000000000000000000000000000009E
:10422000000000000000000000000000000000008E
:10423000000000000000000000000000000000007E
:10424000000000000000000000000000000000006E
:10425000000000000000000000000000000000005E
:10426000000000000000000000000000000000004E
:10427000000000000000000000000000000000003E
:10428000000000000000000000000000000000002E
:10429000000000000000000000000000000000001E
:1042A000000000000000000000000000000000000E
:1042B00000000000000000000000000000000000FE
:1042C00000000000000000000000000000000000EE
:1042D00000000000000000000000000000000000DE
:1042E00000000000000000000000000000000000CE
:1042F00000000000000000000000000000000000BE
:00000001FF
